** EXPERIMENTAL (HLL) ** Open Watcom Linker Version 1.6beta1 Limited Availability
Portions Copyright (c) 1985-2002 Sybase, Inc. All Rights Reserved.
Created on:       13/11/17 16:25:34
Warning! W1121: file U:/tmp\ldconv_pyexpat_obj_1aaf52885a541a3548.obj(U:\DEV\python-2.7.5\Modules\pyexpat.c): '_initpyexpat' has already been exported
Executable Image: build/lib.os2knix-2.7/pyexpat.pyd
creating an OS/2 EMX dynamic link library


                        +------------+
                        |   Groups   |
                        +------------+

Group                           Address              Size
=====                           =======              ====

CGROUP                          0001:00000000        00024bd0
DGROUP                          0002:00000000        000022c0



                        +--------------+
                        |   Segments   |
                        +--------------+

Segment                Class          Group          Address         Size
=======                =====          =====          =======         ====

TEXT32                 CODE           CGROUP         0001:00000000   00024bd0
________TEXT           CODE           CGROUP         0001:00024bd0   00000000
DATA32                 DATA           DGROUP         0002:00000000   000020b0
SET1__os2dll           DATA           DGROUP         0002:000020b0   00000004
SET2__os2dll           DATA           DGROUP         0002:000020b4   00000000
SET3__os2dll           DATA           DGROUP         0002:000020b4   00000004
SET1___CTOR_LIST__     DATA           DGROUP         0002:000020b8   00000004
SET2___CTOR_LIST__     DATA           DGROUP         0002:000020bc   00000000
SET3___CTOR_LIST__     DATA           DGROUP         0002:000020bc   00000004
SET1___DTOR_LIST__     DATA           DGROUP         0002:000020c0   00000004
SET2___DTOR_LIST__     DATA           DGROUP         0002:000020c4   00000000
SET3___DTOR_LIST__     DATA           DGROUP         0002:000020c4   00000004
SET1___crtinit1__      DATA           DGROUP         0002:000020c8   00000004
SET2___crtinit1__      DATA           DGROUP         0002:000020cc   00000000
SET3___crtinit1__      DATA           DGROUP         0002:000020cc   00000004
SET1___crtexit1__      DATA           DGROUP         0002:000020d0   00000004
SET2___crtexit1__      DATA           DGROUP         0002:000020d4   00000000
SET3___crtexit1__      DATA           DGROUP         0002:000020d4   00000004
SET1___eh_frame__      DATA           DGROUP         0002:000020d8   00000004
SET2___eh_frame__      DATA           DGROUP         0002:000020dc   00000014
SET3___eh_frame__      DATA           DGROUP         0002:000020f0   00000004
SET1___eh_init__       DATA           DGROUP         0002:000020f4   00000004
SET2___eh_init__       DATA           DGROUP         0002:000020f8   00000004
SET3___eh_init__       DATA           DGROUP         0002:000020fc   00000004
SET1___eh_term__       DATA           DGROUP         0002:00002100   00000004
SET2___eh_term__       DATA           DGROUP         0002:00002104   00000004
SET3___eh_term__       DATA           DGROUP         0002:00002108   00000004
SET1___fork_parent1__  DATA           DGROUP         0002:0000210c   00000004
SET2___fork_parent1__  DATA           DGROUP         0002:00002110   00000000
SET3___fork_parent1__  DATA           DGROUP         0002:00002110   00000004
SET1___fork_child1__   DATA           DGROUP         0002:00002114   00000004
SET2___fork_child1__   DATA           DGROUP         0002:00002118   00000000
SET3___fork_child1__   DATA           DGROUP         0002:00002118   00000004
________DATA           DATA           DGROUP         0002:00002120   00000000
BSS32                  BSS            DGROUP         0002:00002120   000001a0
c_common               BSS            DGROUP         0002:000022c0   00000000
________BSS            BSS            DGROUP         0002:000022c0   00000000


                        +----------------+
                        |   Memory Map   |
                        +----------------+

* = unreferenced symbol
+ = symbol only referenced locally

Address        Symbol
=======        ======

Module: U:\usr\lib\dll0hi.obj({standard input})
0001:00000000* __text
0002:00000000* __data
0002:00000000* ___data_start
0002:00002120* ___bss_start
0002:000020b0+ __os2dll
0002:000020b8  ___CTOR_LIST__
0002:000020c0  ___DTOR_LIST__
0002:000020c8* ___crtinit1__
0002:000020d0* ___crtexit1__
0002:000020d8  ___eh_frame__
0002:000020f4  ___eh_init__
0002:00002100  ___eh_term__
0002:0000210c+ ___fork_parent1__
0002:00002114+ ___fork_child1__
Module: U:/tmp\ldconv_pyexpat_obj_1aaf52885a541a3548.obj(U:\DEV\python-2.7.5\Modules\pyexpat.c)
0001:0000719b  _initpyexpat
0002:00002120* _template_string
Module: U:\usr\local473\lib\libc_dll.lib(dllinit.obj)
0001:00007f20  _DLL_InitTerm
Module: U:\usr\lib\libend.lib(src/libend/386/endlink386.asm)
0002:000022c0  _end
0002:00002120  _edata
Module: U:\usr\lib\libend.lib(src/libend/386/end.asm)
0001:00024bd0* _etext
0001:00024bd0* __etext
0000:00000000* WEAK$ZERO
0002:000022c0  __end
0002:00002120  __edata
Module: U:\extras\lib\expat.lib(xmlparse.obj)
0001:00007fb3* _XML_UseParserAsHandlerArg
0001:00007fbe  _XML_UseForeignDTD
0001:00007fe8  _XML_SetReturnNSTriplet
0001:0000800c  _XML_SetUserData
0001:00008027  _XML_GetBase
0001:00008035  _XML_GetSpecifiedAttributeCount
0001:00008043* _XML_GetIdAttributeIndex
0001:00008051  _XML_SetElementHandler
0001:00008065  _XML_SetStartElementHandler
0001:00008073  _XML_SetEndElementHandler
0001:00008081  _XML_SetCharacterDataHandler
0001:0000808f  _XML_SetProcessingInstructionHandler
0001:0000809d  _XML_SetCommentHandler
0001:000080ab* _XML_SetCdataSectionHandler
0001:000080bf  _XML_SetStartCdataSectionHandler
0001:000080cd  _XML_SetEndCdataSectionHandler
0001:000080db  _XML_SetDefaultHandler
0001:000080f0  _XML_SetDefaultHandlerExpand
0001:00008105* _XML_SetDoctypeDeclHandler
0001:00008119  _XML_SetStartDoctypeDeclHandler
0001:00008127  _XML_SetEndDoctypeDeclHandler
0001:00008135  _XML_SetUnparsedEntityDeclHandler
0001:00008143  _XML_SetNotationDeclHandler
0001:00008151  _XML_SetNamespaceDeclHandler
0001:00008165  _XML_SetStartNamespaceDeclHandler
0001:00008173  _XML_SetEndNamespaceDeclHandler
0001:00008181  _XML_SetNotStandaloneHandler
0001:0000818f  _XML_SetExternalEntityRefHandler
0001:0000819d* _XML_SetExternalEntityRefHandlerArg
0001:000081b4  _XML_SetSkippedEntityHandler
0001:000081c2  _XML_SetUnknownEncodingHandler
0001:000081d9  _XML_SetElementDeclHandler
0001:000081ea  _XML_SetAttlistDeclHandler
0001:000081fb  _XML_SetEntityDeclHandler
0001:0000820c  _XML_SetXmlDeclHandler
0001:0000821d  _XML_SetParamEntityParsing
0001:00008247  _XML_SetHashSalt
0001:00008271  _XML_StopParser
0001:000082e8* _XML_ResumeParser
0001:000083d1  _XML_GetErrorCode
0001:000083df  _XML_GetCurrentByteIndex
0001:000083fe* _XML_GetCurrentByteCount
0001:00008420  _XML_GetInputContext
0001:00008451  _XML_GetCurrentLineNumber
0001:000084aa  _XML_GetCurrentColumnNumber
0001:00008500  _XML_FreeContentModel
0001:00008515* _XML_MemMalloc
0001:0000852a* _XML_MemRealloc
0001:00008545* _XML_MemFree
0001:0000855a  _XML_ErrorString
0001:0000857f  _XML_ExpatVersion
0001:00008589  _XML_ExpatVersionInfo
0001:000085a7  _XML_GetFeatureList
0001:0000869f* _XML_DefaultCurrent
0001:00008e66  _XML_ParserFree
0001:000092b6* _XML_GetParsingStatus
0001:000092fc  _XML_GetBuffer
0001:0000991f  _XML_SetBase
0001:00009969* _XML_SetEncoding
0001:0000a69f  _XML_ParseBuffer
0001:0000a808  _XML_Parse
0001:0000b4df  _XML_ExternalEntityParserCreate
0001:0000bb72  _XML_ParserCreate_MM
0001:0000bb8e  _XML_ParserCreateNS
0001:0000bbb6  _XML_ParserCreate
0001:0000bbd9* _XML_ParserReset
Module: U:\tmp\ldconv_libgcc_so_d_a_1aaf52885a55182dc0.lib(emx-ctordtor.obj)
0001:000116f0  ___ctordtorInit
0001:00011724  ___ctordtorTerm
Module: U:\extras\lib\expat.lib(xmlrole.obj)
0001:000130c0  _XmlPrologStateInit
0001:000130e3  _XmlPrologStateInitExternalEntity
Module: U:\extras\lib\expat.lib(xmltok.obj)
0001:000220af  _XmlUtf8Encode
0001:0002214f* _XmlUtf16Encode
0001:00022197  _XmlSizeOfUnknownEncoding
0001:000223cc  _XmlInitUnknownEncoding
0001:000228f2  _XmlGetUtf8InternalEncoding
0001:000228fc* _XmlGetUtf16InternalEncoding
0001:00022963  _XmlInitEncoding
0001:00022a55  _XmlParseXmlDecl
0001:00022aa5  _XmlGetUtf8InternalEncodingNS
0001:00022aaf* _XmlGetUtf16InternalEncodingNS
0001:00022b16  _XmlInitEncodingNS
0001:00022c08  _XmlParseXmlDeclNS
0001:00022c58  _XmlInitUnknownEncodingNS
Module: U:\tmp\ldconv_libgcc_so_d_a_1aaf52885a55182dc0.lib(emx-eh.obj)
0001:00024b60  ___ehInit
0001:00024b96* ___ehTerm


                        +----------------------+
                        |   Imported Symbols   |
                        +----------------------+

Symbol                              Module
======                              ======

___libc_ForkRegisterModule          libc065
___init_dll                         libc065
___libc_Back_termDll                libc065
___libc_ForkDeregisterModule        libc065
__atfork_callback                   libc065
_PyArg_ParseTuple                   python27
_Py_BuildValue                      python27
_PyUnicodeUCS2_Decode               python27
_PyInt_FromLong                     python27
_PyObject_GC_UnTrack                python27
_PyObject_GC_Del                    python27
_PyString_FromString                python27
__Py_NoneStruct                     python27
_PyUnicodeUCS2_DecodeUTF8           python27
__Py_ZeroStruct                     python27
__Py_TrueStruct                     python27
_PyList_New                         python27
_PyList_Append                      python27
_Py_FindMethod                      python27
_PyString_FromStringAndSize         python27
_PyErr_NoMemory                     python27
__PyObject_GC_New                   python27
_PyObject_GC_Track                  python27
_PyArg_ParseTupleAndKeywords        python27
__Py_HashSecret                     python27
_PyExc_RuntimeError                 python27
_PyErr_SetString                    python27
_PyExc_TypeError                    python27
_PyExc_ValueError                   python27
_PyDict_New                         python27
_PyTuple_New                        python27
__PyThreadState_Current             python27
_PyEval_GetGlobals                  python27
_PyFrame_New                        python27
_PyEval_CallObjectWithKeywords      python27
_PyErr_Fetch                        python27
_PyTuple_Pack                       python27
_PyErr_Restore                      python27
_PyTraceBack_Here                   python27
_PyObject_CallFunction              python27
_PyObject_SetAttrString             python27
_PyErr_SetObject                    python27
_PyObject_IsTrue                    python27
_PyCode_NewEmpty                    python27
_PyObject_GetAttrString             python27
_PyObject_Call                      python27
_PyErr_Format                       python27
_PyErr_Occurred                     python27
_PyString_AsString                  python27
_PyExc_AttributeError               python27
_PyDict_GetItem                     python27
_PyDict_SetItem                     python27
_PyInt_AsLong                       python27
_PyType_Type                        python27
_Py_InitModule4                     python27
_PyModule_AddObject                 python27
_PyModule_AddStringConstant         python27
_PySys_GetObject                    python27
_PyModule_GetDict                   python27
_PyErr_NewException                 python27
_PyErr_Clear                        python27
_PyModule_AddIntConstant            python27
_PyCapsule_New                      python27
_PyModule_New                       python27
__CRT_init                          libc065
__CRT_term                          libc065
__assert                            libc065
__std_free                          libc065
__std_strcmp                        libc065
__std_malloc                        libc065
__std_sprintf                       libc065
__std_memcpy                        libc065
___ctordtorInit1                    libc065
___ctordtorTerm1                    libc065
__std_memmove                       libc065
__std_memset                        libc065
__std_time                          libc065
__std_srand                         libc065
__std_rand                          libc065
__std_realloc                       libc065
___register_frame_table             gcc473
___deregister_frame                 gcc473


                        +--------------------+
                        |   Libraries Used   |
                        +--------------------+

U:\extras\lib\expat.lib
U:\tmp\ldconv_python2_7_dll_a_1aaf52885a541a7f80.lib
U:\tmp\ldconv_libgcc_so_d_a_1aaf52885a55182dc0.lib
U:\usr\lib\libc_alias.lib
U:\usr\local473\lib\libc_dll.lib
U:\usr\lib\libend.lib


                        +-----------------------+
                        |   Linker Statistics   |
                        +-----------------------+

Stack size:  0000 (0.)
Memory size:  00026e90 (159376.)
Link time: 00:00.10
